:1000000010C015C014C013C012C011C010C00FC062
:100010000EC00DC00CC00BC00AC009C008C007C08C
:1000200006C011241FBECFEDCDBF02D03EC0E8CF29
:100030008AB388698ABB87B3876087BBC19A8FEF11
:1000400094E3ACE081509040A040E1F700C0000094
:10005000DB9A8FEF93EDA0E381509040A040E1F751
:1000600000C00000C29AC09ADB988FEF93EDA0E326
:1000700081509040A040E1F700C00000C198DB9A99
:100080008FEF91E1AAE781509040A040E1F700C0D6
:100090000000C098DB988FE798E3A1E08150904082
:0E00A000A040E1F700C00000F6CFF894FFCFBB
:00000001FF
